:020000000528D1
:080008005729831681171830F7
:100010008500F03086008312850186018B11060869
:100020000B10831687308100831281010B1123206E
:100030001723002993006820FF3903190800462080
:100040001308013E1A2815231523152303308600B3
:1000500005140A23051015230330860005140A230E
:1000600005100F230330860005140A230510023003
:10007000860005140A230510152328305720083060
:100080005720013057200630572008009400D7230E
:10009000140E0F3986008510051505140000051093
:1000A00014080F398600051400000510080094009C
:1000B000D723140E0F398600851005110514000092
:1000C000051014080F3986000514000005100800FB
:1000D0008207543458342034463452344534513431
:1000E0003A34003420342034203420342C3420346A
:1000F00020343034003430343034003400003234B2
:1001000035340034000035343034003400003734E6
:10011000353400340000493432344334203445341B
:10012000723472343A3400346F346E3420346134B3
:10013000643472344334323400346234753473348A
:1001400020346C346F3477342034003450346C34C1
:100150006C3420346F3475347434203400346F348C
:10016000663420346C346F3463346B3420340034A0
:100170005334653474342D347534703420344D3434
:10018000003465346E3475342034563431342E34B2
:10019000323400344634723420344D3469346E3491
:1001A0003A3400344634723420344D346134783477
:1001B0003A340034533474346534703420344C345D
:1001C0006F3400345334743465347034203448341C
:0401D000693400345A
:100200009A019B019D0103133C2246220C3057208A
:10021000861E3C2BC5233C2246228F228B158B1633
:100220008B1720309C009C0803192A299D0803196C
:10023000132906301D020319132901301D02031969
:10024000332902301D0203194B2905301D02031901
:100250003F2913298B139C08031D31292E230530B8
:100260009C008B171329831B3A299B128B13462260
:100270008B1713299B168B1346228B171329831B6D
:1002800046299B138B1346228B1713299B178B131D
:1002900046228B171329831B52291B138B134622CB
:1002A0008B1713291B178B1346228B1713290B1837
:1002B0005C290B196D2909008B1106080B10060823
:1002C000061F7D21861F8621061EC2220B108B155C
:1002D00020309C008101031709008B120B11810152
:1002E0009C03831F782906301D02031D9D0A7B296C
:1002F0009D08031D9D038B1609000F23061B080094
:10030000861B80298F21861B080083290F23861BCB
:100310000800061B89299C21061B08008C29260839
:10032000861E27089E0703189F0AAF211A1CA929B9
:100330009A1CAD29BD2208002608861E27089E02A9
:10034000031C9F03C2211A1CA9299A1CAD29BD2296
:1003500008003C2246228F2208009B220800230826
:1003600092001F089202031CBD29031D08002208E9
:1003700092001E0892020318080021089F0020081E
:100380009E0008001F08920021089202031CD02939
:10039000031D08001E08920020089202031808009E
:1003A00023089F0022089E000800831205080739D1
:1003B00085008316051685150A2305120A230800F1
:1003C0008316051285150A2305160A2383120800D1
:1003D000831685110A2308309600970DFE21960B8F
:1003E000ED298316851105160A2385150A230310A6
:1003F0008312051A0314831685110800031C0512C5
:100400000318051685150A23851108008316851122
:1004100005160A23083096002822970D960B0C2A01
:100420008316851105120A2385150A2308008316F1
:10043000851105160A23083096002822970D960B81
:100440001D2A8316851105160A2385150A2308001F
:1004500085150A2303108312051A031483168511C8
:100460000A2308008030572022301A20C03057203D
:100470002B301A20FD2208001E0898001F08990042
:100480000310980D990DFE3098050800C2309700B2
:10049000D521E8210318322219089700E82118080D
:1004A0009700E821CE309700E8211B089700E8214B
:1004B000E0210800883057203D301A20C8305720EE
:1004C00046301A2008008030572000301A20C030F3
:1004D000572009301A2008008312103093008D0134
:1004E0008E018F01910D900D8F0D8E0D8D0D930B43
:1004F0007A2A00340F30840084220E308400842253
:100500000D3084008422722A033000079200921971
:100510008000303000079200921B8000003463227C
:100520001E0803398C00C530572003108C0D8C0D2C
:100530000C08123E1A201F0890001E08FC3991007A
:100540000310900C910C900C910C6C229301C03014
:1005500057200E0EB2220E08B2220F0EB2220F0842
:10056000B22208000F391318BA2A031DB92AF03035
:10057000BA2A1314303E462008001E0891001F08B6
:100580009000A52A1523061A0800831FCB2A83137F
:10059000061A0800C82A8317C82A1523861A0800D5
:1005A0000000861A0800D12A003089001E08880041
:1005B000F022890A1F088800F0220313080089002E
:1005C0001E08DB2A00308900EC2208089E00890AF8
:1005D000EC2208089F000800831608148312080004
:1005E00083160815081255308900AA30890088142E
:1005F000081EF82A08118312080010309200042304
:100600009203031DFF2A080081010B110B1D062B0D
:100610000B1108000A309500950B0C2B08000A30CE
:1006200092000A23920B112B08009630102B831294
:100630000508073985008316051685150A238312D8
:10064000851D252B051E252B0800803057202230C4
:100650001A20C030572034301A206300031BD422E4
:100660004622C230013E9700D521E8211722E02121
:10067000171B080008000800D323803057204F3094
:100680001A20C030572058301A20861E452B1523BB
:10069000861A482B2930A3006830A2000C30A10034
:1006A0008030A0002830A60001309A00D32380308B
:1006B000572061301A208C010230E3229B22861ED3
:1006C0005F2B1523061F7D21861F8621861A622B2C
:1006D00015230230D522D3238030572069301A20C9
:1006E0008C010430E3229B22861E742B1523061FE7
:1006F0007D21861F8621861A772B15230430D5226B
:10070000A3012830A200A1010130A000A6000330FF
:100710009A00D3238030572071301A208C01083082
:100720008900EC2208089E0091009F019001BD22E3
:10073000861E982B1523061F7D21861F8621861A6B
:100740009B2B15230830DF22D323803057207930AC
:100750001A208C0109308900EC2208089E009100C3
:100760009F019001BD22861EB32B1523061F7D21FC
:10077000861F8621861AB62B15230930DF22023008
:10078000E3220030D5229A010A290B3092001E3054
:10079000840000308900EC2208088000890A840A5D
:1007A000920BCB2B0800013057201523080083162D
:1007B000FF30860083120511851405140510060EFE
:1007C000F03992000514051006080F399204921BA7
:0E07D000D72B85108316F030860083120800A8
:02400E000100AF
:104200009000130080000C006800290000000000EE
:064210000100280001007E
:00000001FF
